:020000040000FA
:10000000092882073F3406345B344F3466346D343C
:100010007D3483160F308500860183128030810085
:100020008601A501A60107309F0044280A30A100DF
:100030000000A00B1828A10B182800340230A200E1
:10004000A00B2028A10B2028A20B20280034A618E2
:100050007728A6140630250603197728A50A7728DD
:10006000A6187728A6140130250603197728003032
:10007000250603197728A5037728A5010120860006
:1000800044288601162067283F3086001E2006304F
:1000900086001E205B3086001E204F3086001E200A
:1000A000663086001E206D3086001E207D30860062
:1000B0001E20A501012086005D28851C3D28051D08
:1000C000652885195D28A50A6728A50A6728851C63
:1000D0003D28051D2720851D30202508012086008C
:1000E00016200519A6108519A610051C4128672899
:02400E00503F21
:00000001FF
